:10000000D0260020550100005101000051010000E0
:1000100000000000000000000000000000000000E0
:10002000000000000000000000000000510100007E
:10003000000000000000000051010000510100001C
:100040005101000051010000510100005101000068
:100050005101000051010000510100001911000080
:100060005101000051010000510100005101000048
:1000700051010000000000000000000051010000DC
:100080005101000051010000510100005101000028
:1000900051010000000000000000000051010000BC
:1000A0005101000051010000510100005101000008
:1000B0000000000010B5064C2378002B07D1054B3B
:1000C000002B02D0044800E000BF0123237010BDC4
:1000D000CC00002000000000E82F0000044B10B509
:1000E000002B03D00349044800E000BF10BDC04608
:1000F00000000000D0000020E82F0000024B034A5F
:100100005A6005221A60704710E000E0FFFFFF0010
:1001100070B580250B0E0C4A0C4CD8B26D0201381C
:10012000C0B2FF280AD118061B1A5B1853609360EF
:1001300080235B0211681942FCD070BD546094604A
:1001400016682E42FCD0EAE710E000E0FFFFFF0057
:10015000FEE700002549264870B581420AD0254BAC
:10016000C41E0022A34203D303331A1A920892003A
:10017000214B98472148224BC11E0022994203D8A7
:1001800003331A1A9208920000211E4B9847FF224F
:100190001D4B032193431D4A0C2593600222082422
:1001A00030261B4B1B485A62C3788B431343C370E2
:1001B000C378AB432343C370174B987BB04306000F
:1001C000202030439873987BA84304439C73987B0A
:1001D000884302439A738023104A51680B4353604B
:1001E0000F4B98470F4B9847FEE7C046E82F00009B
:1001F00000000020CC0000201D260000CC000020C4
:10020000CC0600202F2600000000000000ED00E0DA
:10021000FC70004100500041004800410040004196
:10022000D5250000AD1B0000F0B517000A7885B099
:1002300053060C0001909B0F012B52D16379097971
:100240002A4D1B020B432978994202D069789942C2
:1002500047D1E679A379360252B21E43002A0FDA5B
:100260000020012F0AD06378212B11D1072E3BD11A
:100270000300A91D320001981D4CA04705B0F0BD38
:100280001C4B984763780100202B03D0222B19D0F8
:100290000D2027E0072E27D1002F01D13B00E9E7F1
:1002A0003200154C02A8A0472B69002B05D107226C
:1002B000A81D02A9A0470020E0E702A8984700284F
:1002C000F5D1F8E700230A4E1A0019001800B047CC
:1002D0006B69002BEFD0E078A278000210439847BA
:1002E000E9E70A204042C9E70120FBE7E8000020D7
:1002F00001200000292400001D260000F7B515008C
:1003000001294FD0022900D176E0002900D075E004
:10031000836810681E00009302330193002802D105
:100320000A20404220E00821437982788B43022B47
:10033000F6D133789A4263D0FF2B63D1327069686B
:100340000522324B9847041E0FD1286804220378F7
:100350006968C0182D4B9847019B0136B342DDD127
:10036000012220002A4B5A71FEBD637922791B02BB
:10037000A778D2183800E178264B92B29847002827
:1003800042D17BB2244A002B09DAB770380090477B
:100390002C6020786968214B20189847D3E7009B90
:1003A0001F71F3E78468002A05D0136808225B797F
:1003B0009343022BB4D12378FF2B07D0FF25A078DD
:1003C0002570A84202D0164B9847A5706378FF2B82
:1003D00007D0FF25E0786570A84202D0104B9847FF
:1003E000E5702079FF2803D00D4B9847FF23237138
:1003F0000020074B5871B7E71B2092E70D2090E7CC
:1004000012208EE71C208CE714208AE72D160000AE
:10041000E80000203D190000CD190000471600003B
:10042000A119000010B50A4B984701280CD80948BB
:10043000094B0062C361094B1830984701200849F5
:10044000084B9847002010BD11204042FBE7C046F2
:1004500035240000E8000020FD020000D123000048
:10046000000000204523000010B5074B0A00597911
:100470000400002905D02100D878044C0123A047AE
:1004800010BD11204042FBE7E800002001200000E1
:100490000A0010B5032810D8094B02F03FF80208F3
:1004A0000A0C18790221074B9847002010BDD87814
:1004B000F8E71961F9E75961F7E70D204042F5E7E0
:1004C000E8000020611B0000014B58797047C046CE
:1004D000E8000020054A03001168002901D1044901
:1004E00011601068C31813607047C0460C010020EB
:1004F000D026002000207047074B9A8C920604D526
:100500001022D9681142FCD004E0D021DA680A40F8
:10051000D02AFBD17047C04600080040002803D015
:10052000002901D00230C0B2142301305843014BDE
:10053000C0187047700100200F2370B50100807C47
:10054000072503401A00CC7C083225405B01012DB1
:1005500008D01449520152181021D171124A9B1827
:10056000597270BD40252C4206D08026AC43CC7415
:100570000D4C1C196671A5710825CC7C5201AC4349
:10058000CC7400240949C9188C728C76054952181C
:100590006F21D171044A9B185972054B9B6898478B
:1005A000DFE7C04600500041FF500041100100202D
:1005B0007001002020238B40DAB20F2310B5040015
:1005C000807C054903405B015B185A72034B012193
:1005D0001B69A268984710BDFF50004170010020C0
:1005E00010B50300807CFF2809D04024DA7C224229
:1005F00005D0A243DA74024A14699A68A04710BD74
:1006000070010020F7B59446837C134A01AE0D00BB
:100610003280FF2B1AD04027C27C3A4216D00F22DC
:1006200013401C0008346201002910D00B4FD2196E
:10063000802717710949640164180949725D5B01DB
:100640005B18E27161465A72064B9847F7BD034941
:1006500052185771EEE7C046254A0000005000418D
:10066000FF500041E1050000F0B50D000F21837C33
:1006700085B00B409C46304B03AE338063465B0134
:100680000093634608332D495C01002D20D0095D9D
:100690004906490F009A2C01A418294A765D1419BD
:1006A000A77AFFB2022917D101390F4214D0A77AD5
:1006B000224A5B019B188F43009AA772DE71214B7F
:1006C0002940D218567204221F4B984705B0F0BD3E
:1006D0000C5D07212140DDE702213A000A4001922A
:1006E0000F4217D0A27AC77C8A43A272134A5B01D9
:1006F0009B18DE71009A134BD218072356723B40A9
:10070000012BE3D17B06E1D5C17CC909A942DDD02B
:100710000022D9E7624651004D19094A2D015519A9
:10072000019A5B01AA72054A9B18DE71009A054B7B
:10073000D2185672CAE7C0460408000000500041B3
:1007400010010020FF500041050600008C2370B509
:10075000FF26094D9B00094CED1803212000084B92
:1007600098470021A674E1741434AC42F5D160229C
:10077000044B0548984770BD70010020840100209B
:10078000E10500002F26000010010020F0B50F2722
:1007900085B00191837C040002931F40002399429D
:1007A00005D04B4B7A019B185B699B049B0C258AF7
:1007B000484AAC46954202D06A1E12B294460722BD
:1007C000E07C02400392019A002A04D042497A0157
:1007D00052180221D171A26899186268A1609142F1
:1007E00040D22368521A59187B01394E92B20293B3
:1007F00083062CD52B1C954200D9131C9DB22A00D0
:10080000364BE0689847324BE26879015B181A6111
:100810007B01F6187369AD049B0BAA0C9D0315436D
:10082000756173692E4A13407361019B002B08D1D7
:10083000039B4E22012B00D0043A2A497B015B180E
:100840009A72254A7B019B1880225A7139E08023D5
:10085000151C9B019A4200D91D1C7B01F318ADB2F7
:100860001961D5E710267A0130420ED0E37C1C498D
:10087000B343E374164B9A18921953689B0B9B036E
:10088000536053680B405360CFE7039801281AD197
:10089000144812184B205072624613409D420CD1EE
:1008A0004025E37C0298AB43E3740F4BDB68984729
:1008B000002806D1E37C2B43E374002120000B4B7E
:1008C000984705B0F0BD074812184A20E3E7C04634
:1008D00010010020FF030000005100411D26000010
:1008E000FF3F00F0FF50004170010020E1050000D3
:1008F0000F23F0B5857C85B004000E001D400391E8
:10090000019100290AD0614B6A019B1859680901BD
:100910008A0C0392596889048B0C0193238A0093F3
:10092000009A5B4B9A4203D01300013B9BB20093A9
:10093000019B009FE27C1F40072313400293002E7F
:1009400004D054496B015B180121D97193060FD56E
:100950006368002B0CD0A26821689B1A88181A1CA7
:100960009BB2BB4200D93A1CE1684B4B92B298470C
:1009700063686A019446002B2CD1E27CD10629D50C
:1009800030339A43103B1A43E2746246E1683F4BAE
:1009900042489950218A63445A68890409090240EF
:1009A0000A435A605A68920B92035A60002E0BD188
:1009B000029925226B01012903D1344AD218967677
:1009C0002D2237495B189A72324B6D01ED18402386
:1009D0002B711DE0A168002E1CD0228ABA4219D9C1
:1009E0001022E37C9343E374019B5918A160029A9F
:1009F0006B01012A46D12A4A9B182D225A72002DDA
:100A000002D1224BE2681A6000212000254B984752
:100A100005B0F0BD039A5118A1608B42E7D92020A0
:100A2000E27C5B1A278A9BB2024216D0391C9F4295
:100A300000D9191CE068154A8BB269015050134A5D
:100A40001648624451689B041B0901400B435360E4
:100A500053689B0B9B035360A8E79F420BD28020F7
:100A6000800183420CD8009A93432068074A4118BA
:100A700068011150E3E79F42F7D91043E074F4E7AF
:100A80000300F2E7064A9B182522B7E71001002071
:100A9000FF030000005100411D260000FF3F00F051
:100AA000FF500041E1050000802302009B00072069
:100AB0009A4214D8013BFF3B01389A420FD80138C3
:100AC000802A0CD80138402A09D80138202A06D8B3
:100AD0000138102A03D806309042804140427047C6
:100AE00010B52A4CA378DB0718D40323A2781A4246
:100AF000FCD10222237813420AD023789343237037
:100B00000323A2781A42FCD10223A2781A42FCD114
:100B1000012323700233A2781A42FCD10123A27868
:100B20001A42FCD11A4B1B4A1A605A609A60DA606A
:100B30001A61194B98471F20184B1A68530B910CD8
:100B4000920103400140520F834200D105231F2927
:100B500000D10239072A00D1023A9B010B4312034C
:100B6000134323850323E2781A43E2700C22E178D1
:100B70000A43E27004222270A278100018401A4240
:100B8000FAD1074B63620123238110BD005000415D
:100B900070010020F50400004D0700002460800073
:100BA0001001002003220E4B9978114214D199783C
:100BB0001142FCD102221978C8B2114205D1024378
:100BC0001A70032299781142FCD180210020054A35
:100BD0001160054A1A83704711204042FBE7C04666
:100BE0000050004100E100E08D0200000121024AB6
:100BF00013898B43138170470050004180231843B1
:100C0000014B98727047C04600500041F7B50F2461
:100C100004402E4B00910600C10947B2200001920A
:100C200098470321009B05000B400093022C44D8F9
:100C3000837CFF2B44D1009B002B10D1F943C9B218
:100C4000224B2000C9099847837CFF2B38D1F33B06
:100C500063431F4A9B58002B34D113202EE0002FF2
:100C600014DA0C2262431A4B9B185A68002A19D1D5
:100C70000C236343164CE418636800200099EB6072
:100C8000019B01312B82E974AE74FEBD0C236343DA
:100C90000F4A9B58002B0BD00C2262430C4B9B1825
:100CA0001B8900E05B89019A9A42D6DC002FDFDBCA
:100CB0000C235C43064BE358DFE712204042E4E795
:100CC0001420FBE7002FE7DACBE7C0461D05000044
:100CD000882E0000F7B50F2504000540022D1AD814
:100CE00043B2C70901933900144B28009847837C0D
:100CF0000600FF2B0FD00322114B39009847072223
:100D0000F37C1340012B07D100220E4B0834640101
:100D1000E254FF237382F7BD63B2002B07DA70221F
:100D2000094B6D01ED186B7893436B70F1E7064B3F
:100D30006401E418637893436370EAE71D050000DB
:100D40000506000000500041FF500041F7B50F2498
:100D50000440C109474B45B220009847464B61010A
:100D6000CE1872780700D2B2022C00D97DE0837CC5
:100D70000193FF2B00D178E0404B5C18C37C072126
:100D80001800084001283BD1772311001940009139
:100D90001A4200D06CE0663B73703D8A384B2800E5
:100DA0009847E023374ADB0500071840AB031340A0
:100DB00003436360402180230F22AD04AD0C284320
:100DC0006061B1717371009B2C48A372A376019B83
:100DD000AC031340FA685B011A50C01842682A4DF0
:100DE0001540254345604268920B92034260224AB7
:100DF00000989B18B0225A71A03A99719A72FEBD60
:100E0000002D19DA702115000D400A4230D15B0720
:100E10005B0E134373703F8A194B38009847E023E9
:100E20000007DB0518408023BF04BF0C3843606116
:100E30007371A5762800E2E715000D400A4217D12C
:100E40005B075B0F134373703F8A0D4B3800984765
:100E50000C4ABB031340E0220007D20510400343B5
:100E600063604023B371A572E4E712204042C6E7F5
:100E70001420FBE71D050000FF5000411001002079
:100E8000A90A000000C0FF0FFF3F00F0F8B50700FF
:100E90000F26C40937400D0038002100294B984720
:100EA0000200022F4AD8837C10203340A040012D3D
:100EB00010D1254D5901C0B2491948712021A140D6
:100EC00022485B01C9B21B1899720823D17C0B43DD
:100ED000D37409E05B01002D29D11D495D181B4920
:100EE0005B18D979084201D100201CE02021A140E3
:100EF000C0B25871C8B258721E7A314204D0012172
:100F0000A140C9B2187259710721D37C1940012937
:100F10000AD1FF35EC792F31200008400C42E3D193
:100F200028398B43D374F8BD08218B43D0E7064A98
:100F30009B189B791840431E9841F4E712204042C9
:100F4000F1E7C0461D05000000510041FF5000417F
:100F500000500041F8B50F231840114B44011B19F4
:100F60000F0019685D68AD04AD0C022812D8002F7F
:100F700010D00C4BE4186378112B0ED11026227A76
:100F80000020324205D008223800074B984728003D
:100F90002672F8BD12204042FBE71320FBE7C04653
:100FA00010010020FF5000411D260000F0B50F2564
:100FB000077A87B07BB23D40FF09390002930600F3
:100FC0003A4B280098473A49038A04001A008B429A
:100FD00001D05A1E92B271680A400192022D62D865
:100FE00080203268800582420DD3324D8818A84295
:100FF00009D8032015000540024204D1029A002AB4
:101000000EDB994206D2E3680125002B08D113209C
:10101000404217E0019B002B16D0E368002B42D022
:10102000E37C02201B070DD4234B05A89847E17CE5
:1010300040230A001A400392204A194206D005A80C
:101040009047012007B0F0BD019DE9E70B43E37431
:1010500005A890477F213368FA0123607368039FD6
:101060006360039BA360E37C0B40134369011D0095
:1010700020239D430D43E574737A002B02D0019F1A
:101080007B425F411022E37C3F0193431F43029B5D
:1010900000212000E774002B03DA094B9847002059
:1010A000D0E7084BFAE71220B2E7C0461D05000062
:1010B000FF030000FF7F00204924000057240000A8
:1010C0008D070000F1080000002900D10549012822
:1010D00002D1054B596070470028FCD1024B1960C2
:1010E000F9E7C046F504000070010020002900D196
:1010F0000749002802D1074B99607047012802D1A7
:10110000044BD960F9E70228F7D1024B1961F4E7E3
:10111000F504000070010020F7B56C4B1A8C91B2F9
:101120000191002A00D066E09A8B198B04200A40B6
:1011300011000140024204D09883654B1B68984718
:10114000F7BD80241600A400264022421DD0614A2B
:101150009A839A82923AFF3A1A835F4B1A8912074E
:10116000120F032A05D01A8D1207120F032A07D176
:101170000121002249015B1819891A814904490D8E
:101180000320534B5B689847DAE78024150025401D
:10119000224205D09C834E4B310005205B68F2E76C
:1011A00070261400344032420AD04A4A9E839E82FE
:1011B0001A834A4B9847464B290002205B68E2E7B6
:1011C0000825110029402A420CD0454A5470414A52
:1011D0009D839E821A83434B98473D4B21000120FB
:1011E0005B68D0E7D20706D53A4A9A839A821E8373
:1011F000374B5B68C7E700260F2701253A4CA37CD5
:10120000FF2B38D02A003B409A400199114232D03E
:1012100036495A01521832495B015B181278997AA3
:101220000B001340114226D014217143284A521852
:1012300047211032D27D1140012911D1DA0603D5A0
:1012400020002B4B984716E0402219001140134212
:1012500001D0290001E09B060DD52000254B09E0B7
:1012600051B200291CDA5906F3D4190708D5290010
:101270002000214B9847013614341B2EBFD15FE765
:10128000990703D5290020001C4BF3E707210A40EA
:10129000012AF0D100215A07EAD4DB06EBD5CFE7CB
:1012A000202019000140034201D00021D5E7580752
:1012B000DED42B4203D029002000114BDAE70721AE
:1012C0000A40012AD7D11A07E7D5D0E700500041DC
:1012D000700100200102000010010020F90400004C
:1012E000FF5000414D0700008401002007510041DC
:1012F00039050000B5050000690600008D070000F3
:10130000F108000010B5024B1860024B984710BD61
:1013100060040020FD000000044B10B51C68044B65
:1013200098470100034B2000984710BD600400203F
:10133000D913000011010000064B1A7AD2B21A72BA
:101340005A7AD2B25A729A7AD2B29A72DA7AD2B2FD
:10135000DA72704700040040064B10B55A685A60B4
:10136000054B9847054B9847054B9847FF20054B81
:10137000984710BD004000413913000025140000BB
:1013800065140000D91500000068002800D17047DE
:101390008842F9D10120FAE770B50C4B05000C002A
:1013A00006689847012358404F22094B0949C0B2AB
:1013B00098472B68002B02D12C60236070BD33004E
:1013C0003668002EFBD11C602660F7E78913000009
:1013D000E1130000AC2E0000FA235B015843704774
:1013E000002800D100BE704710B5054B054898474E
:1013F000054B9847054B06489847064B984710BD44
:10140000712300006404002025040000E92300008B
:10141000080000201D24000010B5014B984710BDA6
:10142000E91300000D4B186A196A890F8A070C49E5
:1014300001400A4302210A431A629A6911439961E1
:101440001F211A7F0A401A771E39DA68D2080A4229
:10145000FBD08022196A0A431A62704700080040D4
:101460000000FF0F02220121144B9A84DA6812094E
:101470000A42FBD0124ADA62FC22D2019A629B2213
:1014800052009A849A8C92080A4210D01022D9688D
:101490001142FCD08022998C0A430A499A844A78E6
:1014A000D209FCD102219A698A439A6170470121CD
:1014B000DA6812090A42FBD0ECE7C0460008004097
:1014C00080BB0104000C0040F8B506000D001400BC
:1014D000002804D0081E02D01000431E9841F122BB
:1014E0001049114B98473700083738000F4B984781
:1014F0000028F8D000263800A95D0D4B9847380029
:101500000A4B98470028FAD00136B442F3D8012597
:10151000002C00D025003800064B98470028FAD050
:101520002800F8BDCA2E0000E11300004B1E000089
:101530003D1E0000551E0000F7B505001400019186
:10154000002804D0081E02D01000431E98418622B5
:101550000C490D4B5200984700262F0008373800E1
:101560000A4B98470028F8D0094B38009847019B50
:1015700098550136B442F0D80120002C00D020004C
:10158000FEBDC046CA2E0000E11300005F1E000031
:10159000431E000070B504000D00002802D00800B2
:1015A000431E98410749084B3422984720002900E0
:1015B000064B08309847002803D1054B6360054B64
:1015C000236070BDCA2E0000E1130000111E000050
:1015D00039150000C9140000C30709D58023104A3B
:1015E0005B00936083235B0253605378DB09FCD17B
:1015F000030708D504230A4AFF339360094B53605D
:101600005378DB09FCD1030608D50823044AFF33CD
:101610009360054B53605378DB09FCD17047C0469B
:10162000000C0040030301000707210010B58842A9
:1016300001D3002010BD0378012BFAD944789442DD
:10164000F8D0C018F3E7884201D300207047037830
:10165000012BFAD94278042AF7D0052AF6D0C0180F
:10166000F1E7000070B50D4B150002220C00984701
:1016700000280FD170BD0378012B0DD94378022BC0
:101680000AD14379AB42F5D0C278837812029B1815
:101690009BB2C018A042EED30020EBE72D1600004D
:1016A00070B50C0016000025A04201D3002070BDCB
:1016B00003222100054B98470028F8D00378012B1E
:1016C000F4D9B542F3D0C0180135EDE72D1600006E
:1016D00002000F21002030B5094B11405C78944284
:1016E0000CD01D78002D01D18C4207D00130C4B23E
:1016F000203340B20D2CF1D10120404230BDC04614
:10170000A40400200020704770B5084B04000D00B1
:101710009847074B40011B189A780020032A03D1F1
:10172000290020009B69984770BDC046D116000073
:10173000A4040020F0B5374B87B00F000090019251
:101740009847354D4401002F41D12E19F770295D7E
:10175000002933D12200B4780C327078F369AA18CA
:10176000032C27D10C270131F757984703007078D5
:10177000002B0BD0294B7380002F02DB863BFF3BF5
:1017800018430121264B984707B0F0BD042203936C
:10179000B2700493002F0ADB8023184302AB187346
:1017A000012302AA537303A81E4B9847ECE70F23AB
:1017B0001840F3E798470223B370E5E70123B370BD
:1017C0002C19E178E369019A00989847DCE72B1916
:1017D000012F0CD10222DA70295D002904D19A7000
:1017E00000980F4B9847EBE705229A70E8E7022F25
:1017F00008D10422DA702A5D002A01D19F70C3E764
:101800000122F2E7032F03D1A022D2005A80D7E7AA
:10181000054AFBE7D1160000A404002005020000E1
:101820008D0E0000AD0F000006060000F7B5184B46
:101830000400984747013B00164D0C335B19190013
:1018400001932000144B98478026C0B2264300968F
:10185000124E082806D001212000B047012100982F
:10186000B047F7BDED19012700212000B047002146
:101870000098B047200001996B69AF709847002825
:10188000EFD1052339002000AB70B0473900E6E7FF
:10189000D1160000A4040020550F00008D0E00009A
:1018A00070B5124B984700281EDBD022104C002147
:1018B0002000104B520098472300FF210D240E4AB0
:1018C000013CE4B259705A619A61DA612033002C0C
:1018D000F6D10A4D20000A49A84701200949A84726
:1018E00002200949A847200070BDC046E10A000057
:1018F000A40400202F26000005170000ED100000B2
:101900002D180000091700003517000010B5014B15
:10191000984710BDC910000010B5014B984710BD85
:10192000A50B000010B5014B984710BDED0B000052
:1019300010B5014B984710BDFD0B0000F8B5104CD9
:1019400006000D001700A047002813DAFF20A0476B
:10195000041E12DB3A00290030000A4B9847002889
:1019600007DB03210020084B64011A190D40567053
:10197000E554F8BD14204042FBE71520FBE7C046C4
:10198000D11600000D0C0000A4040020002110B5A9
:1019900002000800014B984710BDC0463D190000E9
:1019A00070B5074B05009847041E07DB2800054B60
:1019B0009847FF23044864010419637070BDC04652
:1019C000D1160000D50C0000A404002070B50C4B0B
:1019D0000400984700280FDB0A4D4001425D2D1896
:1019E00051424A4101322000074BAA709847002813
:1019F00001DA0023AB7070BD12204042FBE7C04605
:101A0000D1160000A40400204D0D0000F0B5037AAB
:101A100004008BB018000193324B9847637A061E7E
:101A2000656802935BDB304B06A89847730100930F
:101A3000009A2E4B9E18B37804AAD71D3B703A78B3
:101A4000D3B203932A4B012A1DD10232B27006A8E9
:101A50009847264B009AD35C002B1FD00298019B1D
:101A6000421E9041D909C0B22368227A0793089593
:101A7000002931D080231A4304AB1A7558751D4BC9
:101A800007A8984708E006A898473B780120DAB2F3
:101A9000062B01D8184B98560BB0F0BDF27CB37CE6
:101AA00012029B189BB2002B05D1042203981D0043
:101AB0000100B270D8E79D4200D91D000B490020FB
:101AC0008C46009A01006244127B7F2ACCD99D4249
:101AD0009B4101315842C7E70F231A40CCE712203F
:101AE0004042D9E7D116000049240000A404002098
:101AF00057240000AD0F0000E62E0000F8B50500E9
:101B00000E1E1AD1124B9847041E1DDB022128001D
:101B1000104FB84700280FD031002800B8470028E0
:101B20000ADB0D480D4B6401241863803200032149
:101B30002800E36998473000F8BD064B012900D022
:101B4000022128009847F7E712204042F4E7C046F8
:101B5000D11600008D0E0000A40400200103000037
:101B600070B50F4B14000D009847002C00D10D4CA0
:101B7000002809DB012D08D0022D0BD0002D03D148
:101B8000094B40011818446170BD074B40011818FB
:101B90008461F9E7044B40011818C461F4E7C046BA
:101BA000D116000005170000A404002010B5044B56
:101BB0009847044B98470448044B9847FEE7C046B3
:101BC000691E00007D240000F42E0000C9240000DE
:101BD00030B501240C4BC5B2C0180378CAB2A34378
:101BE0000A49234303706B085B180F2019782542BC
:101BF00005D0014012011143C9B2197030BD8143B3
:101C00000A431A70FAE7C04640440041304400419C
:101C100010B51620034C0449A04717200349A047DC
:101C200010BDC046D11B00000200160002001700C4
:101C30002023044A116A0B431362034B034A5A8060
:101C40007047C04600040040000C004017400000F0
:101C500010B5054B984700220449054B05489847A5
:101C6000054B984710BDC046311C000000140042CF
:101C70009515000044060020111C000010B5024814
:101C8000024B984710BDC04610E000E0051300006D
:101C9000F8B5C02580238027114C124AED05FF05B9
:101CA0005B04AB60A762A262220004266B6158321B
:101CB00013781820B34313700B490C4B98478023BB
:101CC0000B4A9B04AB60A762A2626B615934237814
:101CD0001920B34323700749044B9847F8BDC04609
:101CE00000440041000100C006001800D11B0000A4
:101CF000000200C0060019002022064BD9690A43E1
:101D0000DA61402259690A435A61034B034A5A80F7
:101D10007047C04600040040000C00400647000029
:101D200010B5034B9847034B9847034B984710BD9A
:101D3000F91C0000A1180000911C000010B5044B14
:101D40009847044B9847044B9847044B984710BD5D
:101D500059130000511C00007D1C0000211D0000D3
:101D6000C3691942FCD17047022210B503680321F0
:101D700093430360014B984710BDC046611D0000AE
:101D80001B4B70B5C3189B0ADBB20400032B04D0B5
:101D90000020184A1849194B9847E369184DDB078A
:101DA00011D4022603212000A8472368334205D01E
:101DB0002000144B984731002000A8470523032139
:101DC00020002360A84720000121A8470E4B2000D7
:101DD00023600321A847C0239B02200063600721E2
:101DE000A8470020094BA381A0733034207070BD38
:101DF00000F8FFBD3A020000002F0000E1130000D0
:101E0000611D0000691D00000400104004C5FFFFB3
:101E100070B50500431E98410C00B4220449054BDF
:101E2000C0B298472C602000034B984770BDC04655
:101E3000002F0000E1130000811D000003681985D8
:101E400070470368188DC0B270470368187E01237D
:101E5000184070470368187E8007C00F70470368FA
:101E6000187E4007C00F704710B5024B9847024BD1
:101E7000984710BD3D1D000019140000064B10B519
:101E80001C69002C00D110BD2000636800220121D4
:101E900098472468F5E7C0465006002070B5050055
:101EA0000E00064BDC68002C00D170BD6368002B6F
:101EB00002D03100280098472468F4E7500600203B
:101EC000F8B505000E0017000B4B9C68002C01D1E3
:101ED0002000F8BD6368002B01D12468F6E73A00C2
:101EE000310028009847002804D00A30F5D001209E
:101EF0004042EEE70120ECE750060020054B10B50C
:101F00005C68002C00D110BD6368002B00D098479E
:101F10002468F6E75006002010B51400002903D00D
:101F2000012923D0002010BD1378002BFAD153785B
:101F3000052B0FD0092BF5D1E17892780E4B0902D1
:101F40001143D9764A1E91410331997601200B4BFA
:101F50009847E7E70A4B90789847E178A27809021A
:101F600011434B1E9941044B0231EEE70A00054B29
:101F7000210000209847D5E7500600209D1E000054
:101F800031190000C11E000070B5002402260C4B60
:101F900098470C4D20006E830B4B6C7798470B4B8A
:101FA000287F98470A4D210020000A4AA84731009F
:101FB0002000094AA8472000084B984770BDC0463A
:101FC0007D1E000050060020A11900008D190000A0
:101FD000611B00001D200000191F0000CD1900002A
:101FE00010B5002802D0012803D010BD024B98473D
:101FF000FBE7024B9847F8E79D1E0000891F000091
:102000001FB502926A461073537301A8024B0191E7
:10201000984705B000BDC0460D1A0000F7B5B74B94
:10202000002204000D009847030000205A1C00D134
:10203000C1E00130834200D1BDE02B781F2219009E
:10204000914304D0802900D1B6E00020B3E0687845
:1020500001380A28F9D800F057FA46F856F80BF874
:10206000F8F806F86000AA78002A0BD1A44B98472C
:102070000022012311002000A24CA04743425841F6
:10208000C0B298E0A04D2B6803CBA04B9847002826
:1020900000D190E0C37881781B02C91889B2411839
:1020A00004229B4B01919847FF220090009B002B3C
:1020B000DED09E78964202D02F69002F0AD1009878
:1020C000042203780199C0180090914B9847320080
:1020D0000090EBE76A46002138007B6898470028AB
:1020E000EDD03F68E9E7022BAFD1EE79AB7936024C
:1020F0001E43AAD131002879864B9847012332002C
:102100003100200054E0022B9FD1EB79AE791B0205
:102110001E439AD101212879EEE7EC78AB782402AE
:102120001C432B796D79784E2D021D433368F27E66
:1021300003CB764B9847002887D004220090C378C1
:1021400081781B02C91889B24118714F0191B847B3
:10215000002800D179E78378AB4210D1C378A3423D
:102160000DD137690090002F00D16EE701216A463A
:1021700038007B689847011E08D03F68F3E7009855
:10218000042203780199C0180090E0E76A463800FD
:102190007B689847002800D057E7002C04D0012224
:1021A000AA40737F1343737700231A0019001800A5
:1021B000544CA0470120FEBD68780A2800D944E7A6
:1021C00000F0B6F9620043FF43FF43FF43FF43FFC4
:1021D0000B0043FF5A0043FF8300E978AB78090204
:1021E0000B43090ACAB2022917D0032A34D00020AF
:1021F000012AE0D1AB79ED792D021D43424B1B68DA
:1022000003CB434B9847011E00D11EE72A1C122D19
:1022100000D91222002392B22DE7AA79ED79013379
:102220002D021543384A1068167F03C8DAB2374BBF
:102230009847011E00D108E7C37882781B02D218A4
:1022400092B20023954205D9013E35406B425D4173
:10225000EBB215002A000EE7AA79ED792D0215439D
:10226000294A1068167F03C8DAB22B4B9847011E23
:1022700000D1EAE60278E4E72349CB7E4A6913708D
:102280004969002301223CE71F211E221800194042
:10229000104013420ED0022900D0D6E61D4B2879FB
:1022A000984703000020834200DA84E701300340AE
:1022B000009300E00090144D02226946174B6869B4
:1022C00098470023022269691BE70F4E6B79297931
:1022D000727F1B020B431A4101241000204022424E
:1022E0001ED03469002C00D1AFE62A000221200064
:1022F0006368984700281BDA2468F3E7C11E0000D2
:102300007D1E000001200000500600206516000020
:102310002D160000FD1A0000A11600001D26000069
:1023200073692200187071690300054DA84741E7E1
:1023300073690122187000237169180038E7C046DC
:102340000120000010B5012808D0022809D000287B
:1023500003D105480430054B984710BD02480830AA
:10236000F9E701480C30F6E7500600209913000009
:1023700070B50400431E98410C4A0D4B0D49C0B284
:1023800098470D4B984700280EDB0C4D20220C4B34
:1023900000212800984700200A496C610A4CA04798
:1023A00001200A49A047002070BDC0465503000027
:1023B000E11300001B2F0000A118000050060020B0
:1023C0002F260000FD1E00000D190000E11F000077
:1023D00010B501000248034B1030984710BDC046AD
:1023E000500600209913000010B50A4B9C7E002C6B
:1023F0000BD100280CD002681860D2791A7701221C
:102400009A76054B9847200010BD04204042FBE718
:102410000920FBE7500600201919000010B5014BF8
:10242000984710BD25190000014B58697047C046F8
:1024300050060020034B987E1023184200D018004D
:102440007047C04650060020EFF31083036072B659
:10245000BFF35F8F7047BFF35F8F036883F310880C
:1024600070470000012382B0034201D0024A13707A
:10247000002002B07047C0467006002010B50B4C1B
:102480000B4B40220021201D98470A4B98470A4BCE
:1024900098470028FBD003200849094B9847237828
:1024A000002BFCD0074B6420984710BD700600201D
:1024B0002F26000019140000C90400006524000044
:1024C00091040000191300000FB413B50A4C04AABC
:1024D00002CA043400922000084B9847084B2000A1
:1024E0009847084B0100200098470190002016BC37
:1024F00008BC04B01847C0467006002079260000CA
:102500003F2600006904000002B4714649084900F2
:10251000095649008E4402BC7047C04602B4714659
:1025200049084900095C49008E4402BC7047C04616
:1025300003B47146490840004900095E49008E44D1
:1025400003BC7047002934D00123002210B4884214
:102550002CD301242407A14204D2814202D20901D2
:102560001B01F8E7E400A14204D2814202D24900F3
:102570005B00F8E7884201D3401A1A434C08A04296
:1025800002D3001B5C0822438C08A04202D3001B2C
:102590009C082243CC08A04202D3001BDC08224343
:1025A000002803D01B0901D00909E3E7100010BC83
:1025B000704701B5002000F00BF802BD0029F8D0EB
:1025C00003B5FFF7C1FF0EBC4243891A1847C04646
:1025D0007047C04670B500260C4D0D4C641BA4100E
:1025E000A64209D1002600F0EFFC0A4D0A4C641BFC
:1025F000A410A64205D170BDB300EB589847013630
:10260000EEE7B300EB5898470136F2E7D42F00000D
:10261000D42F0000D42F0000D82F0000002310B5C5
:102620009A4200D110BDCC5CC4540133F8E70300DA
:102630008218934200D1704719700133F9E70023E3
:10264000C25C0133002AFBD1581E704700B59BB015
:10265000009104910649059102910649039169464A
:1026600000F0D8F80023009A13701BB000BDC046DC
:10267000FFFFFF7F0802FFFF10B513000A000100F3
:1026800002480068FFF7E2FF10BDC0466800002066
:1026900070477047F8B50323CD1C9D4308350600ED
:1026A0000C2D1FD20C25A9421ED8300000F064FB6F
:1026B00025490A681400002C1AD1244F3B68002BCE
:1026C00004D12100300000F027FB386029003000E1
:1026D00000F022FB431C2BD10C233000336000F0B0
:1026E00053FB03E0002DDEDA0C2333600020F8BD3D
:1026F00023685B1B19D40B2B03D92360E4182560D6
:1027000003E06368A2420ED10B60300000F03CFB96
:10271000200007220B30231D9043C21A9842E6D0B6
:102720001B1AA350E3E75360EFE722006468C2E797
:102730000323C41C9C43A042E1D0211A300000F0C6
:10274000EBFA431CDBD1C7E7B4060020B806002033
:10275000F0B58E6885B007000C00039201939E428D
:102760003CD890238A89DB001A4234D003250969BA
:1027700023685B1A0293636902985D43EB0F5D194E
:10278000019B6D1001331B18AB4200D91D0053058E
:1027900032D529003800FFF77DFF061E09D10C2332
:1027A0003B6040230120A28940421343A38105B02E
:1027B000F0BD029A2169FFF731FFA389144A1A403C
:1027C00080231343A381029B2661F618266065616E
:1027D000019EED1AA560019B9E4200D9019E320028
:1027E0000399206800F0B5FAA36800209B1BA36042
:1027F00023689E192660DAE72A00380000F016FBED
:10280000061EE0D13800216900F0C6FAC7E7C046CD
:102810007FFBFFFFF0B5A1B003901D008B890F0077
:1028200016001B0611D50B69002B0ED14021FFF7B6
:1028300031FF38603861002805D10C23039A013834
:10284000136021B0F0BD40237B61002308AC6361BD
:10285000203363761033A376079535002B78002B51
:1028600001D0252B47D1AB1B0593B5420CD03200CC
:1028700039000398FFF76CFF431C00D1AEE062699A
:10288000059B9446634463612B78002B00D1A5E03F
:10289000012200235242626004A9543252186E1C75
:1028A0002360E360A3601370A36505223178544868
:1028B00000F044FA751C00281FD12268D30604D505
:1028C000532304A95B1820211970130704D553233F
:1028D00004A95B182B21197033782A2B16D03500E8
:1028E00000210A20E3682A786E1C303A092A4ED962
:1028F000002911D117E00135B0E7414B2268C01A19
:102900000123834013432E002360CEE7079B191D4C
:102910001B680791002B01DB0B9304E05B42E36033
:102920000223134323602B782E2B0AD16B782A2B9A
:1029300035D1079B02351A1D1B680792002B2BDB34
:102940000993304E03223000297800F0F7F900286F
:1029500006D04023801B8340226801351343236047
:102960002978062228486E1C217600F0E7F9002815
:102970003CD0264B002B25D10722079B07339343DE
:10298000083307936369049A9B18636165E74343BF
:10299000350001219B18A6E701235B42D0E7002305
:1029A0000A201A000135636029786E1C3039092924
:1029B00003D9002BC5D00992C3E742433500012358
:1029C0005218F1E707AB00933A002100104B03982F
:1029D00000E000BF0490049B0133D3D1BB890D9864
:1029E0005B0600D42DE7012040422AE707AB0093A5
:1029F0003A002100064B039800F07CF8EAE7C04655
:102A0000942F00009A2F00009E2F0000000000006D
:102A100051270000F7B5150001938A680B690C0077
:102A20000090934200DA130022002B6043321278A8
:102A3000002A01D001332B6023689B0602D52B6846
:102A400002332B602268062317001F401A4227D04A
:102A5000230043331B785A1E93412268920630D4D8
:102A6000220001990098089E4332B047431C25D0AC
:102A7000062320682A68E16800250340042B03D15F
:102A80008D1AEB43DB171D40A3682269934201DDD9
:102A90009B1AED180027BD4220D1002010E001371D
:102AA000E3682A689B1ABB42D2DD22000123019908
:102AB0000098089E1932B047431CF0D101204042D3
:102AC000FEBD3020E1184331087021005A1C453109
:102AD0000978A218433202331170C1E722000123A2
:102AE00001990098089E1A32B047431CE6D001377E
:102AF000D1E70000F0B58BB006920A00433207938D
:102B0000059004920A7E0C00109B782A06D8622A4F
:102B100008D8002A00D1C0E0582A52D026004236F8
:102B2000327022E0100063381528F7D8FFF700FD57
:102B300016001F00F6FFF6FFF6FFF6FF1F00F6FF78
:102B4000F6FFF6FFF6FFA80036009A00F6FFF6FF44
:102B5000B900F6FF3600F6FFF6FF9E0026001A6861
:102B60004236111D1960136833700123A7E008680D
:102B700019680A1D05060BD50D681A60002D03DAC9
:102B80002D23049A6D421370614B0A27039332E0A0
:102B90000D681A604106F1D52DB2EFE70D6819688E
:102BA000081D18602E0601D50D6803E06D06FBD5E3
:102BB0000D68ADB2564B0A2703936F2A17D1082729
:102BC00015E045310A70524A03921A68216820CAFA
:102BD0001A60080650D5CB0702D52023194321607F
:102BE0001027002D03D1202322689A43226023005E
:102BF000002243331A706368A360002B03DB0422B6
:102C0000216891432160002D02D1049E002B0CD03D
:102C1000049E28003900FFF7D1FC039B013E5B5C5A
:102C200033702B0005009F42F3D9082F09D1236888
:102C3000DB0706D563682269934202DC3023013E3C
:102C40003370049B9B1B2361079B21000093059815
:102C5000069B09AAFFF7DEFE431C35D10120404246
:102C60000BB0F0BD202209680A43226022007821BF
:102C700045321170274AA7E74806ACD5ADB2AAE79E
:102C80001A680D68101D4969186013682E0601D571
:102C9000196002E06D06FBD519800023049E2361B4
:102CA000D2E71A68111D19601668002130006268A9
:102CB00000F044F8002801D0801B60606368236145
:102CC0000023049A1370BFE7236932000699059820
:102CD000079DA847431CC1D023689B0715D4099BB7
:102CE000E0689842BCDA1800BAE72200012306998E
:102CF0000598079E1932B047431CAFD00135E368F1
:102D0000099A9B1AAB42F0DCE9E70025F7E7C046D9
:102D1000A52F0000B62F0000002370B5064D04005B
:102D200008002B60FDF7D6FB431C03D12B68002B5A
:102D300000D0236070BDC046C8060020C9B282180A
:102D4000904201D10020704703788B42FBD00130C4
:102D5000F6E710B5884202D98B18984203D30023B6
:102D600007E08B5C8354013AFBD210BDCC5CC454A9
:102D700001339A42FAD1F8E710B50248FFF788FC10
:102D800010BDC046C006002010B50248FFF781FC08
:102D900010BDC046C006002070B50500002910D047
:102DA0000C1F2368002B00DAE4182800FFF7E4FF6B
:102DB0001D4A1368002B05D1636014602800FFF7DB
:102DC000E3FF70BDA34208D9216860188342F3D1A4
:102DD00018685B6841182160EEE71A005B68002BF9
:102DE00001D0A342F9D911685018A0420BD1206834
:102DF0000918501811608342E0D118685B684118C7
:102E000011605360DAE7A04202D90C232B60D5E7AA
:102E100021686018834203D118685B6841182160FB
:102E200063605460CAE7C046B4060020F8B50700E6
:102E30000D001600002905D11100FFF72BFC04003E
:102E40002000F8BD002A03D1FFF7A6FF3400F7E702
:102E500000F012F82C00B042F2D231003800FFF737
:102E600019FC041EECD029003200FFF7D7FB290023
:102E70003800FFF791FFE3E70B1F1B68181F002BBB
:102E800001DA0B58C0187047200400200000000031
:102E900040000000E00300200000000040000000AF
:102EA000A003002000000000400000002E2E2F682C
:102EB000616C2F7574696C732F7372632F757469ED
:102EC0006C735F6C6973742E63002E2E2F68616CB7
:102ED0002F7372632F68616C5F75736172745F73B7
:102EE000796E632E6300ED0101010102F0ED000136
:102EF000010102F048656C6C6F20576F726C6400C2
:102F00002E2E2F68706C2F736572636F6D2F687033
:102F10006C5F736572636F6D2E63002E2E2F757359
:102F2000622F6465766963652F75736264632E63CF
:102F30000000000000000000000000000000000091
:102F40000000000000000000000000000000000081
:102F50000000000000000000000000000000000071
:102F60000000000000000000000000000000000061
:102F70000000000000000000000000000000000051
:102F80000000000000000000000000000000000041
:102F900000000000232D302B2000686C4C0065667B
:102FA000674546470030313233343536373839419A
:102FB00042434445460030313233343536373839B0
:102FC0006162636465660000F8B5C046F8BC08BC81
:102FD0009E467047DD000000F8B5C046F8BC08BC4E
:082FE0009E467047B500000099
:102FE80000000000290200001000002065000020F9
:102FF8001201000202000040EB030424000100005B
:1030080000010902430002010080320904000001A6
:103018000202000005240001100524010100042417
:10302800020205240600010705820340000A09047C
:103038000100020A00000007050102400000070520
:1030480081024000000000006C0000200000000029
:10305800542F0000742F0000342F000000000000DF
:103068000000000000000000000000000000000058
:103078000000000000000000000000000000000048
:103088000000000000000000000000000000000038
:103098000000000000000000000000000000000028
:0C30A8000000000000000000000000001C
:00000001FF
